:04000000803117280C
:100008007E1480310B1D09280A2815280B117A083F
:10001800F400F5017408F0007508F100803124201F
:1000280080317E100900803119288531BF25803143
:10003800FA00F901CB01CC017E1020008231C32ADD
:100048000130F2007208F90779080139F3007308E2
:100058002000B000F11B312832283F287108803A6F
:10006800F20080307202031D3B280B307002031C23
:100078003E283F2841282000B0010A30700671044C
:1000880003194728482852287003710403194D287A
:100098004E2852282000A001A1015A28200030082B
:1000A800F200F3017208A0007308A100200C2200DE
:1000B800031C8D1303188D170A3070067104031979
:1000C80066286728722802307006710403196D28A3
:1000D8006E2872282000A201A3017A282000300887
:1000E800F200F3017208A2007308A300220C220098
:1000F800031C8E1303188E170A3070067104031937
:1001080086288728922803307006710403198D28E1
:100118008E2892282000A401A5019A2820003008E2
:10012800F200F3017208A4007308A500240C220051
:10013800031C0E1303180E170A30700671040319F6
:10014800A628A728B2280430700671040319AD2820
:10015800AE28B2282000A601A701BA28200030083E
:10016800F200F3017208A6007308A700260C22000B
:10017800031C8E1103188E150A30700671040319BA
:10018800C628C728D2280530700671040319CD285F
:10019800CE28D2282000A801A901DA28200030089A
:1001A800F200F3017208A8007308A900280C2200C5
:1001B800031C0E1003180E140A307006710403197C
:1001C800E628E728F2280630700671040319ED289E
:1001D800EE28F2282000AA01AB01FA2820003008F6
:1001E800F200F3017208AA007308AB002A0C22007F
:1001F800031C0C1103180C150A307006710403193E
:1002080006290729122907307006710403190D29D8
:100218000E2912292000AC01AD011A29200030084E
:10022800F200F3017208AC007308AD002C0C220038
:10023800031C8C1003188C140A30700671040319FF
:1002480026292729322908307006710403192D2917
:100258002E2932292000AE01AF013A2920003008AA
:10026800F200F3017208AE007308AF002E0C2200F2
:10027800031C0C1003180C1408002000BA003108E5
:1002880032040319482949299A293A08023E860066
:100298008701403FB300413FB4003A088600870118
:1002A800403FB500413FB6003608803AB7003408F1
:1002B800803A3702031D622933083502031865297D
:1002C8006629E22920003A08860087010230810762
:1002D80041310318810A3A0886008701403FB3007C
:1002E800413FB4003A08043E86008701403FB5000C
:1002F800413FB6003608803AB7003408803A3702E2
:10030800031D88293308350203188B298C29E22913
:1003180020003A08063E860087013A08083E840015
:100328008501403F803F413F813FE2293A088600EE
:100338008701403FB300413FB4003408803AB5001C
:1003480080303502031DAA2901303302031CAD2970
:10035800AE29E22920003A0886008701FE3081078D
:100368004131FF30813D7F313A08063E86008701E2
:10037800403FB300413FB4003A0886008701403F40
:10038800B500413FB6003608803AB7003408803AD5
:100398003702031DD129330835020318D429D5297A
:1003A800E22920003A08043E860087013A08083E00
:1003B80084008501403F803F413F813F20003A084B
:1003C80086008701403FB300413FB4003A08083E29
:1003D80086008701403FB500413FB6003608803AA5
:1003E800B7003408803A3702031DFC293308350268
:1003F800031CFF29012A0130022A00302000B8001E
:10040800B9013808B1003908B20008002000C1005D
:10041800C9180F2A112A0130122A0030BC00BD0168
:100428003C08B1003D08B2003B08813141218231CE
:1004380020003208C0003108BF003F084004031DF7
:10044800262A272A392A4108860087010108031924
:100458002E2A2F2AC22A4108860087010330010666
:10046800031D372A382A392AC22A3F0840040319AB
:100478003E2A3F2A752A4108860087010108031988
:10048800462A472A502A4108860087010330010678
:10049800031D4F2A502A542A41088531A825823144
:1004A80020004108860087018101810A4108043E35
:1004B80086008701160001040319632A642A6B2A3F
:1004C8004108043E860087010030C03FC13F410813
:1004D800023E860087010230810741310318810AF4
:1004E800C22A0230BC004108860087013C0881000E
:1004F8004108023E86008701160001040319852A77
:10050800862A942A4108023E860087010030C03FAF
:10051800C13F0130BC00410A860087013C088107C1
:100528004108043E860087010230810741310318E3
:10053800810A4108043E86008701403FBC00413FD4
:10054800BD003D08803ABE0080303E02031DAE2A41
:10055800C9303C02031CB12AB22AC22A0330200047
:10056800BC004108860087013C0881004108063E1E
:10057800860087012030C03F0330C13F0800843126
:100588006D248231B630853162258231B6308531AD
:10059800A8258231AC308431DF248231A230853104
:1005A8000C25823185319A258231E8302000B1004E
:1005B8000330B2007608023EB3000030773DB40045
:1005C8008331D223823120003208F7003108F60047
:1005D800A23085318225823120003B083C04031972
:1005E800F62AF72A0B2B22000E12FF302000C80033
:1005F8004808FA00B6308531A8258231003020003D
:10060800B100B200AC30853139258231442B8431B8
:10061800A924823184312624823120003208210025
:10062800A100200031082100A0002008210403199E
:100638001E2B1F2B252B20082000C8004808FA0075
:10064800442BAC302000C8004808C200B6308331C3
:1006580063238231200043082100A10020004208C2
:100668002100A000200A031D3E2B210A03193D2B5F
:100678003E2B3F2B1F2BFF302000C8004808FA00F4
:1006880006302000C8003030890B482BC80B482B97
:10069800000020004C08803AC800A7304802031D1B
:1006A800572B10304B0203185A2B5B2BD62A0230DB
:1006B8002000CB070030CC3DD62A803117282000F7
:1006C800C7004C08803AC40081304402031D6E2BD9
:1006D800F4304B020318712B722B782BFF3020005B
:1006E800C200FF30C300D12B20004208C4004408D8
:1006F800BB00470882310A22833120004708860060
:10070800870103300106031D8A2B8B2B722B4708A8
:10071800063E86008701403FC400413FC5004508AA
:10072800803AC60080304602031D9C2B01304402EB
:10073800031C9F2BA02B722B20004708063E860027
:100748008701FE3081074131FF30813D7F31470805
:10075800063E86008701403FC400413FC50045086A
:10076800803AC60080304602031DBC2B013044028B
:100778000318BF2BC02BC62B200047088531A8259E
:100788008331722B2000470A860087010108C400C4
:10079800C5014408C2004508C30008002000B7018D
:1007A800B41FD72BD82BDF2BB309B409B30A03190D
:1007B800B40AB701B70AB21FE22BE32BE82BB10941
:1007C800B209B10A0319B20A310832040319ED2B30
:1007D800EE2B172CB601B60AFA2B0130B135B20D43
:1007E800890BF22B0130B5003508B607B21FFD2B77
:1007F800FE2BF12B32083402031D042C310833027E
:10080800031C072C082C0C2C3108B3023208B43B0B
:100818000130B236B10C890B0D2C0130B602031D24
:10082800162C172CFE2B370803191B2C1C2C212CDB
:10083800B309B409B30A0319B40A3408B200330877
:10084800B10008002000C91A2A2C2B2C2E2CB1012B
:10085800B2016C2C4919312C332C0130342C003066
:10086800B300B401B335B40DB335B40DB335B40D1D
:10087800781A3F2C412C0130422C0030B500B601CB
:10088800B535B60DB535B60DF81A4B2C4D2C0130D3
:100898004E2C0030B700B801B735B80D781B552C71
:1008A800572C0130582C0030B900BA0137083904E8
:1008B800BB0038083A04BC0035083B04BD003608C4
:1008C8003C04BE0033083D04B10034083E04B200C5
:1008D8000800210095131908873970389900991371
:1008E8001908FC390238990038308C003830240057
:1008F8008C00703021008D00703024008D0026306F
:1009080021008E00263024008E0023008C018D01EA
:100918008E0121009D0126008C018D018E01200091
:100928008C018D018E018B170B178B160B11210073
:1009380095121512951104302000B1000030B20054
:100948008531B42584318B1708002000B201B20A22
:100958007708803AB10080303102031DB52C9730FA
:100968007602031CB82CB92CD72C7708803A2000C3
:10097800B10081303102031DC32C2C307602031CD8
:10098800C62CC72CD52C7708803A2000B1008130BE
:100998003102031DD12CC3307602031CD42CD52C74
:1009A800D72C2000B2012000320C2200031C0E12AA
:1009B80003180E1608002000B100310886008701D0
:1009C8000030C03FC13F3108023E860087010F302A
:1009D800C03F0030C13F3108043E860087010A301D
:1009E800C03F0030C13F3108063E86008701043011
:1009F800C03F0030C13F3108043E860087013108FE
:100A0800083E84008501403F803F413F813F080008
:100A18002000B1003108860087010030C03FC13F87
:100A28003108023E86008701C830C03F0030C13F10
:100A38003108043E860087019630C03F0030C13F30
:100A48003108063E860087015030C03F0030C13F64
:100A58003108043E860087013108083E840085017C
:100A6800403F803F413F813F08002000B5003508E6
:100A7800860087013108C03F3208C13F310832047F
:100A88000319472D482D512D3508063E860087014C
:100A9800403FB300413FB400592D3508043E86005D
:100AA8008701403FB300413FB4003508083E860047
:100AB80087013308C03F3408C13F08002000B10057
:100AC8003108860087018101310A8600870181018A
:100AD8003108023E860087010030C03FC13F31081F
:100AE800043E860087010030C03FC13F3108063E02
:100AF800860087010030C03FC13F08002000BF00CA
:100B0800CA19872D892D01308A2D0030BD00BE01FC
:100B18003D08B1003E08B2003F08813141218531CE
:100B280020003208BC003108BB00080020000C0877
:100B3800B1003108CA000D08B1003108F8000E08EC
:100B4800B1003108C90008002000B300330885311E
:100B580062258531FF302000B2003208FA00080013
:100B68002100150820003106F839310621009500CA
:080B7800080002340034FF34D0
:020000040001F9
:04000E00A4C9FFDEA4
:00000001FF
